:1000000012C01895189599C01895189518951895B7
:100010001895189518951895189518951895189578
:100020001895189518950FED0DBF00E009BF01B99F
:1000300008E008B900E001B908E808B927E027BBE3
:1000400022E021BB0BEE08BB0FE302BB00E00093F4
:1000500060000093610000936200009363000093CE
:1000600064000093650000936600009367000093AE
:1000700068000093690000936A0000936B0000938E
:100080006C0000936D0000937000AED2ADD2ACD284
:100090001DD000E002BD0FBD01E40EBD8FD095D292
:1000A00000916500009369000091660000936A006A
:1000B0009BD28BD295D0A2D20091650000936900AB
:1000C0000091660000936A0079D0F2CF00E002BD93
:1000D0000FBD0BE40EBD0AE70BBD02E10ABD08B778
:1000E000086008BF08B7006408BF08B703FFFDCF6A
:1000F00000E00DBD0CBD08B7086008BF00916200AC
:100100000F5F00936200009163000F4F0093630044
:1001100008B703FFFDCF009162000F5F00936200FC
:10012000009163000F4F0093630008B706FD04C001
:1001300008B7086008BFECCF089500916400003054
:10014000A9F400E00DBD01E10CBD009160000F5F5E
:1001500000936000009161000F4F0093610001E087
:100160000093640008B7086008BF1895009160000C
:100170000F5F00936000009161000F4F00936100DA
:1001800000916200109160000117009163001091CE
:100190006100010739F704B50093650005B50093C8
:1001A000660000E00093640001E000936D0000E051
:1001B000009360000093610009BFD4CF00E001BB51
:1001C00091980DBD0CBD8199FECF0CB500936700D1
:1001D0000DB50093680002E001BB919A6DD00895BF
:1001E000009165001091690001170091660010915F
:1001F0006A00010721F400E0009370000895009167
:10020000690010916500011700916A001091660065
:10021000010748F10091690000936B0000916A00AA
:1002200000936C0000916B0010916500011B00931E
:100230006B0000916C0010916600010B00936C0044
:1002400000916B0010916E00011700916C001091ED
:100250006F00010720F400E000937000089501E0B2
:100260000093700008950091650000936B00009169
:10027000660000936C0000916B0010916900011BF7
:1002800000936B0000916C0010916A00010B0093C9
:100290006C0000916B0010916E00011700916C00D2
:1002A00010916F00010720F400E0009370000895A2
:1002B00002E00093700008950AE5109167000117AD
:1002C00000E010916800010708F01AC20EE61091D4
:1002D0006700011700E010916800010708F009C2EB
:1002E00002E810916700011700E010916800010713
:1002F00008F0F8C106E910916700011700E01091BD
:100300006800010708F0E7C10AEA109167000117C9
:1003100000E010916800010708F0D6C10EEB1091C3
:100320006700011700E010916800010708F0C5C1DF
:1003300002ED10916700011700E0109168000107BD
:1003400008F0B4C106EE10916700011700E01091AB
:100350006800010708F0A3C10AEF109167000117B8
:1003600000E010916800010708F092C10EE01091C2
:100370006700011701E010916800010708F081C1D2
:1003800002E210916700011701E010916800010777
:1003900008F070C106E310916700011701E01091A9
:1003A0006800010708F05FC10AE4109167000117B7
:1003B00001E010916800010708F040C10EE51091BE
:1003C0006700011701E010916800010708F03DC1C6
:1003D00002E710916700011701E010916800010722
:1003E00008F0DEC006E810916700011701E01091E7
:1003F0006800010708F0CDC00AE9109167000117F5
:1004000001E010916800010708F0BCC00EEA1091ED
:100410006700011701E010916800010708F0ABC008
:1004200002EC10916700011701E0109168000107CC
:1004300008F09AC006ED10916700011701E01091D5
:100440006800010708F089C00AEE109167000117E3
:1004500001E010916800010708F078C00EEF1091DC
:100460006700011701E010916800010708F060C003
:1004700002E110916700011702E010916800010786
:1004800008F04FC006E210916700011702E01091DA
:1004900068000107F8F50AE310916700011702E010
:1004A00010916800010778F50EE4109167000117BC
:1004B00002E010916800010708F041C002E61091C7
:1004C0006700011702E010916800010708F06FC093
:1004D00006E710916700011702E01091680001071C
:1004E00008F06CC00AE810916700011702E0109153
:1004F0006800010708F0B0C002E000936E0000E061
:1005000000936F0008950AE000936E0000E00093EE
:100510006F0008950CE000936E0000E000936F0000
:1005200008950EE000936E0000E000936F000895C0
:1005300000E100936E0000E000936F00089508E072
:1005400000936E0000E000936F00089502E10093B5
:100550006E0000E000936F00089504E100936E00C8
:1005600000E000936F00089506E100936E0000E044
:1005700000936F00089508E100936E0000E000937F
:100580006F0008950AE100936E0000E000936F0091
:1005900008950CE100936E0000E000936F00089551
:1005A0000EE100936E0000E000936F00089506E0F6
:1005B00000936E0000E000936F00089504E0009344
:1005C0006E0000E000936F000895789408B708600B
:1005D00008BF08E009BF00916D00013009F0FBCFB2
:1005E00000E000936D00089505E0F02E80E593ECA7
:1005F00081509040E9F7FA94C9F70895009170008E
:10060000003031F400E000BF03BFC19AC09A0895E2
:1006100000917000023049F0C19AC09802E306BF11
:1006200002E400BF05E003BF0895C09AC1980FEF30
:1006300006BF02E400BF05E003BF089502E2009395
:100640006E0000E000936F00089500E200936E00DA
:1006500000E000936F00089503E000936E0000E057
:1006600000936F00089504E200936E0000E0009391
:100670006F00089506E200936E0000E000936F00A3
:10068000089508E200936E0000E000936F00089563
:100690000AE200936E0000E000936F0008950CE200
:1006A00000936E0000E000936F0008950EE2009347
:1006B0006E0000E000936F00089500E300936E0069
:1006C00000E000936F00089502E300936E0000E0E5
:1006D00000936F00089504E300936E0000E0009320
:1006E0006F00089506E300936E0000E000936F0032
:1006F000089508E300936E0000E000936F000895F2
:0E0700000AE300936E0000E000936F0008957E
:00000001FF
